:100000004528B400142020082104031940283A2070
:1000100084133408800664000D280E28A00A0319F2
:10002000A10F0B2880064028FF3A8417800540283E
:10003000A301A200FF30A207031CA307031C402852
:100040000330A100DF3026201A28A101E83EA000DD
:10005000A109FC30031C2F28A00703182C28A00797
:100060006400A10F2C2820183528A01C3928000076
:1000700039280800A009A109A00A0319A10A08004B
:1000800083130313831264000800831686158610F9
:100090000611061083122030BA000330BB0006118F
:1000A000831606118312061083160610831286101B
:1000B00083168610831286193D14861D3D106F2805
:1000C00086193D14861D3D10640003013D18013E54
:1000D000BD18013C031D6F286430182060283D18AE
:1000E000BD143D1CBD106400BD187A286400BD1C01
:1000F000802860283030BC00E530B800B901852880
:100100003030BC00E530B800B90106108316061087
:100110008312BB1A8614BB1E86100530A000A101F5
:1001200006308400043001203B1A86143B1E8610E2
:100130000530A000A1010630840004300120BB1965
:100140008614BB1D86100530A000A1010630840076
:10015000043001203B1986143B1D86100530A00099
:10016000A1010630840004300120BB188614BB1C9A
:1001700086100530A000A101063084000430012063
:100180003B1886143B1C86100530A000A1010630E8
:10019000840004300120BA1B8614BA1F8610053073
:1001A000A000A10106308400043001203A1B86140F
:1001B0003A1F86100530A000A101063084000430EB
:1001C0000120BA1A8614BA1E86100530A000A101BB
:1001D00006308400043001203A1A86143A1E861034
:1001E0000530A000A1010630840004300120BA19B6
:1001F0008614BA1D86100530A000A10106308400C7
:10020000043001203A1986143A1D86100530A000EA
:10021000A1010630840004300120BA188614BA1CEB
:1002200086100530A000A1010630840004300120B2
:100230003A1886143A1C86100530A000A101063039
:10024000840004300120B9188614B91C86100530CA
:10025000A000A10106308400043001203918861462
:10026000391C86100530A000A1010630840004303E
:100270000120B81B8614B81F86100530A000A1010C
:100280000630840004300120381B8614381F861085
:100290000530A000A1010630840004300120B81A06
:1002A0008614B81E86100530A000A1010630840017
:1002B00004300120381A8614381E86100530A0003C
:1002C000A1010630840004300120B8198614B81D3D
:1002D00086100530A000A101063084000430012002
:1002E00038198614381D86100530A000A10106308B
:1002F000840004300120B8188614B81C861005301C
:10030000A000A101063084000430012038188614B2
:10031000381C86100530A000A1010630840004308E
:1003200001203C1B86143C1F86100530A000A10153
:100330000630840004300120BC1A8614BC1E8610CE
:100340000530A000A10106308400043001203C1AD1
:1003500086143C1E86100530A000A10106308400E2
:1003600004300120BC198614BC1D86100530A00085
:10037000A10106308400043001203C1986143C1D84
:1003800086100530A000A101063084000430012051
:10039000BC188614BC1C86100530A000A1010630D4
:1003A0008400043001203C1886143C1C8610053063
:1003B000A000A101063084000430012086148316B9
:1003C000861083120530A000A1010630840004309D
:1003D000012086108316861083123230A000A101FE
:0E03E000063084000130012060286300F529FA
:02400E006D3F04
:00000001FF
